BL51 BANKED LINKER/LOCATER V5.03                                                        10/31/2008  13:23:21  PAGE 1


BL51 BANKED LINKER/LOCATER V5.03, INVOKED BY:
C:\KEIL\C51\BIN\BL51.EXE .\OUT\STC_EEPROM.obj, .\OUT\main.obj TO .\OUT\STC_EEPROM PRINT (.\LST\STC_EEPROM.m51) RAMSIZE (
>> 256)


MEMORY MODEL: SMALL


INPUT MODULES INCLUDED:
  .\OUT\STC_EEPROM.obj (STC_EEPROM)
  .\OUT\main.obj (MAIN)
  C:\KEIL\C51\LIB\C51S.LIB (?C_STARTUP)
  C:\KEIL\C51\LIB\C51S.LIB (?C_INIT)


LINK MAP OF MODULE:  .\OUT\STC_EEPROM (STC_EEPROM)


            TYPE    BASE      LENGTH    RELOCATION   SEGMENT NAME
            -----------------------------------------------------

            * * * * * * *   D A T A   M E M O R Y   * * * * * * *
            REG     0000H     0008H     ABSOLUTE     "REG BANK 0"
            DATA    0008H     0002H     UNIT         _DATA_GROUP_
            IDATA   000AH     0074H     UNIT         ?ID?MAIN
            IDATA   007EH     0001H     UNIT         ?STACK

            * * * * * * *   C O D E   M E M O R Y   * * * * * * *
            CODE    0000H     0003H     ABSOLUTE     
            CODE    0003H     008CH     UNIT         ?C_C51STARTUP
            CODE    008FH     0053H     UNIT         ?PR?MAIN?MAIN
            CODE    00E2H     003EH     UNIT         ?C_INITSEG
            CODE    0120H     0023H     UNIT         ?PR?_ISP_READ_BYTE?STC_EEPROM
            CODE    0143H     0023H     UNIT         ?PR?_ISP_PROGRAM_BYTE?STC_EEPROM
            CODE    0166H     001BH     UNIT         ?PR?READ?MAIN
            CODE    0181H     001BH     UNIT         ?PR?WRITE?MAIN
            CODE    019CH     0017H     UNIT         ?PR?_ISP_ERASE_SECTOR?STC_EEPROM
            CODE    01B3H     0015H     UNIT         ?PR?_DELAY2?MAIN



OVERLAY MAP OF MODULE:   .\OUT\STC_EEPROM (STC_EEPROM)


SEGMENT                                    DATA_GROUP 
  +--> CALLED SEGMENT                    START    LENGTH
--------------------------------------------------------
?C_C51STARTUP                            -----    -----
  +--> ?PR?MAIN?MAIN
  +--> ?C_INITSEG

?PR?MAIN?MAIN                            0008H    0001H
  +--> ?PR?_ISP_ERASE_SECTOR?STC_EEPROM
  +--> ?PR?WRITE?MAIN
  +--> ?PR?READ?MAIN
  +--> ?PR?_DELAY2?MAIN

?PR?WRITE?MAIN                           0009H    0001H
BL51 BANKED LINKER/LOCATER V5.03                                                      10/31/2008  13:23:21  PAGE 2


  +--> ?PR?_ISP_PROGRAM_BYTE?STC_EEPROM

?PR?READ?MAIN                            0009H    0001H
  +--> ?PR?_ISP_READ_BYTE?STC_EEPROM



SYMBOL TABLE OF MODULE:  .\OUT\STC_EEPROM (STC_EEPROM)

  VALUE           TYPE          NAME
  ----------------------------------

  -------         MODULE        STC_EEPROM
  C:0000H         SYMBOL        _ICE_DUMMY_
  D:0090H         PUBLIC        P1
  D:00B0H         PUBLIC        P3
  D:00E8H         PUBLIC        P4
  D:00E6H         PUBLIC        ISP_TRIG
  B:00A8H.7       PUBLIC        EA
  D:00A8H         PUBLIC        IE
  C:019CH         PUBLIC        _isp_erase_sector
  D:00B8H         PUBLIC        IP
  C:0143H         PUBLIC        _isp_program_byte
  D:00E5H         PUBLIC        ISP_CMD
  D:00E3H         PUBLIC        ISP_ADDRH
  D:0098H         PUBLIC        SCON
  D:0088H         PUBLIC        TCON
  D:00E4H         PUBLIC        ISP_ADDRL
  C:0120H         PUBLIC        _isp_read_byte
  D:00E0H         PUBLIC        ACC
  D:00E7H         PUBLIC        ISP_CONTR
  D:00C8H         PUBLIC        T2CON
  D:00E2H         PUBLIC        ISP_DATA
  D:00D0H         PUBLIC        PSW
  -------         PROC          _ISP_READ_BYTE
  D:0004H         SYMBOL        add
  -------         DO            
  D:0007H         SYMBOL        addh
  D:0006H         SYMBOL        addl
  D:0007H         SYMBOL        rdata
  -------         ENDDO         
  C:0120H         LINE#         14
  C:0124H         LINE#         15
  C:0124H         LINE#         18
  C:012AH         LINE#         19
  C:012BH         LINE#         20
  C:012CH         LINE#         21
  C:012EH         LINE#         22
  C:0130H         LINE#         23
  C:0132H         LINE#         24
  C:0135H         LINE#         25
  C:0138H         LINE#         26
  C:013BH         LINE#         27
  C:013EH         LINE#         28
  C:013EH         LINE#         29
  C:0140H         LINE#         31
  C:0142H         LINE#         32
BL51 BANKED LINKER/LOCATER V5.03                                                      10/31/2008  13:23:21  PAGE 3


  C:0142H         LINE#         33
  -------         ENDPROC       _ISP_READ_BYTE
  -------         PROC          _ISP_PROGRAM_BYTE
  D:0002H         SYMBOL        add
  D:0005H         SYMBOL        dat
  -------         DO            
  D:0007H         SYMBOL        addh
  D:0006H         SYMBOL        addl
  -------         ENDDO         
  C:0143H         LINE#         34
  C:0147H         LINE#         35
  C:0147H         LINE#         37
  C:0149H         LINE#         38
  C:014FH         LINE#         40
  C:0150H         LINE#         41
  C:0151H         LINE#         42
  C:0153H         LINE#         43
  C:0155H         LINE#         44
  C:0157H         LINE#         45
  C:015AH         LINE#         46
  C:015DH         LINE#         47
  C:0160H         LINE#         48
  C:0163H         LINE#         49
  C:0163H         LINE#         51
  C:0165H         LINE#         52
  -------         ENDPROC       _ISP_PROGRAM_BYTE
  -------         PROC          _ISP_ERASE_SECTOR
  D:0007H         SYMBOL        num
  -------         DO            
  D:0007H         SYMBOL        addh
  D:0006H         SYMBOL        addl
  -------         ENDDO         
  C:019CH         LINE#         53
  C:019CH         LINE#         54
  C:019CH         LINE#         57
  C:019DH         LINE#         58
  C:019DH         LINE#         59
  C:019DH         LINE#         60
  C:01A0H         LINE#         61
  C:01A2H         LINE#         62
  C:01A4H         LINE#         63
  C:01A7H         LINE#         64
  C:01AAH         LINE#         65
  C:01ADH         LINE#         66
  C:01B0H         LINE#         67
  C:01B0H         LINE#         69
  C:01B2H         LINE#         70
  -------         ENDPROC       _ISP_ERASE_SECTOR
  -------         ENDMOD        STC_EEPROM

  -------         MODULE        MAIN
  C:0000H         SYMBOL        _ICE_DUMMY_
  D:0080H         PUBLIC        P0
  D:0090H         PUBLIC        P1
  D:00A0H         PUBLIC        P2
  D:00B0H         PUBLIC        P3
  D:00E8H         PUBLIC        P4
BL51 BANKED LINKER/LOCATER V5.03                                                      10/31/2008  13:23:21  PAGE 4


  D:00A8H         PUBLIC        IE
  D:00B8H         PUBLIC        IP
  C:0166H         PUBLIC        read
  C:01B3H         PUBLIC        _delay2
  C:008FH         PUBLIC        main
  C:0181H         PUBLIC        write
  D:0098H         PUBLIC        SCON
  D:0088H         PUBLIC        TCON
  I:000AH         PUBLIC        data_buf
  I:0044H         PUBLIC        read_buf
  D:008EH         PUBLIC        AUXR
  D:00C8H         PUBLIC        T2CON
  D:00D0H         PUBLIC        PSW
  -------         PROC          MAIN
  -------         DO            
  D:0008H         SYMBOL        m
  -------         ENDDO         
  C:008FH         LINE#         22
  C:008FH         LINE#         23
  C:008FH         LINE#         25
  C:0092H         LINE#         26
  C:0097H         LINE#         27
  C:009AH         LINE#         28
  C:009DH         LINE#         31
  C:009DH         LINE#         32
  C:009DH         LINE#         33
  C:00A0H         LINE#         34
  C:00A0H         LINE#         35
  C:00AEH         LINE#         36
  C:00AEH         LINE#         37
  C:00B5H         LINE#         38
  C:00B8H         LINE#         39
  C:00BBH         LINE#         40
  C:00C3H         LINE#         41
  C:00CBH         LINE#         42
  C:00CDH         LINE#         44
  C:00CDH         LINE#         45
  C:00D4H         LINE#         46
  C:00D7H         LINE#         48
  -------         ENDPROC       MAIN
  -------         PROC          READ
  -------         DO            
  D:0009H         SYMBOL        m
  -------         ENDDO         
  C:0166H         LINE#         52
  C:0166H         LINE#         53
  C:0166H         LINE#         55
  C:0169H         LINE#         57
  C:0177H         LINE#         58
  C:0180H         LINE#         60
  -------         ENDPROC       READ
  -------         PROC          WRITE
  -------         DO            
  D:0009H         SYMBOL        m
  -------         ENDDO         
  C:0181H         LINE#         62
  C:0181H         LINE#         63
BL51 BANKED LINKER/LOCATER V5.03                                                      10/31/2008  13:23:21  PAGE 5


  C:0181H         LINE#         66
  C:0184H         LINE#         68
  C:0192H         LINE#         70
  C:019BH         LINE#         72
  -------         ENDPROC       WRITE
  -------         PROC          _DELAY2
  D:0006H         SYMBOL        x
  -------         DO            
  D:0005H         SYMBOL        y
  -------         ENDDO         
  C:01B3H         LINE#         74
  C:01B3H         LINE#         75
  C:01B3H         LINE#         77
  C:01BDH         LINE#         78
  C:01BFH         LINE#         79
  C:01C5H         LINE#         80
  C:01C7H         LINE#         81
  C:01C7H         LINE#         82
  -------         ENDPROC       _DELAY2
  -------         ENDMOD        MAIN

Program Size: data=127.0 xdata=0 code=456
LINK/LOCATE RUN COMPLETE.  0 WARNING(S),  0 ERROR(S)
